:10000000080C2500D00C02006607040A6606060AE2
:1000100061006607090A01022E00220C8E00030609
:10002000040A1A0C8E000306180A200CE501040AC3
:10003000D70C0200580289019C014306820A7C0009
:10004000690068007E007F007A00BA023F0C06005B
:10005000300C24006A00A3050509A30443062B0AFB
:100060000F0220003F0C84013F0E43063A0AA4020F
:10007000AA022B0A12024306010DFF0FA40432004C
:10008000A40513024306010DFF0F7500A4043300FD
:10009000090C2400820A0802E20100080008000896
:1000A000000802080308050807080A080D081208D6
:1000B00016081C08220829083008380841084A0890
:1000C00054085F086A087608830890089E08AD08FF
:1000D000BC08CC08DC08ED08FF08090C2E00400025
:1000E00003042F000F032D030306CC01EE02710A57
:1000F0002C002C032D032C032D032C032D032C0388
:100100002D0300080400FF0C2D002E002F00090C09
:1001100024000B0C3D007F0047040000B109470696
:10012000980AD2096606C70567066B06980A46054F
:10013000FC0C3F024306A80ADF01FD02A40A0306E5
:10014000110BBD0200008B0ADF020306F30B8B0AC2
:10015000000000000000C706BF02C704FE038C0AAF
:10016000260A66070008BF027E004705D209660717
:100170000008BF0200001C02890138007802A706AF
:10018000CA0AE7074B09E7064B0929004704DF03C2
:10019000B10A260A00000000000000000000000074
:1001A0000000C60AC103E40A09029C004306000BD2
:1001B0000306DD0ABC021202E00AFC0013028705F6
:1001C0002100000000000008FA02F10A06052605D9
:1001D0001C02000000000000000000000000000001
:1001E00000081A029C000706FB0A0000030606042A
:1001F0000307060500080306260403072605000872
:100200008704000000000000000000000000000063
:100210000008100C8400070E4306F20BC706BF024D
:10022000150B090C3D00A4027F004704C704B10967
:100230004706210BD2096606C70567066106210B32
:100240004604FC0C3F024306090BDF01FD026B0B69
:100250000306110B0A028B018C018D018E018F01A7
:100260004307DC0B6A026B026C026D026E02D2095C
:10027000E400080C0600A4050A02EA07590B9801DD
:100280004307520B0B0299014307520B2C0C24001D
:10029000B407520B2706520BA3054F0A510B270632
:1002A000820A650B0A02F00E700F4307820AA3054B
:1002B000F00A43064E0BB407900143064F0B1A0297
:1002C0007F0E2704430727058A014307520B2B0C97
:1002D0002400A3054F0A00006003DF02140BF50B96
:1002E00088061602930B3E0243067F0B9E00800B8E
:1002F00011023D023F0743060706E706730B96000F
:100300002C0003042C03180CEC01030C88002D00B6
:100310006D09090CAD0011020307700B000000000D
:10032000CD010306160229006B0017024306CE0B0F
:100330007F0E2A00F7079F0B040C8800A20B4802CF
:100340001F0E00002E008E076E06BD0B2F00430609
:10035000AE0B03042A032B03EE02AA0B4F02070E77
:100360002E004306B70B00000000EE02B30B17028D
:100370007F0E2F000A028F00CE0B8A03070ECA01E0
:100380002C00070C8E002D006D090D022F002C0390
:100390002D032C032D03CD008F008A00F707D70B08
:1003A000C901030729000000A705A404820A8900E7
:1003B00003062900D40B000000000000000000002C
:1003C000D209000000000000000000000000000052
:1003D00000000000820A0000000000000000000091
:1003E0000000000000000000000000000000DB0B27
:10040000840C2700310A800C060A830C2700A00CFC
:10041000C6042900080C2800E6046903C604030684
:10042000C6050000E605E8020C0A0000E60400002C
:10043000C60500000000E605C606E704E604E70777
:10044000470A07020F0EE2012B0A2E0A470A2B0A5F
:10045000310A360A470AA7020A02090AA7020F024E
:10046000090AE605C605A702A10C080AC605000090
:10047000E605080C2800E6050305C60703046F031C
:10048000E604C605E8023B0AE6050000E604C604E9
:10049000E6054A0A4B0AC605E7070008010880037B
:1004A0002F000F03070EE2017B0AD70B8D0B950B74
:1004B0005F0B570BF90B3A0B2400070C4C01720928
:1004C0008C07690A6C062001FF0F6C0760010402AB
:1004D000020B400143066F0A6C06250BF90B6C07F3
:1004E000250BF90BE20101080208040808081008AE
:1004F000200840088008A006CA0B0003070EE2018E
:10050000B10BF90BF90BBC0BF90BC30BF90BF90B86
:100510008007B10A0706940A5406960A1F07860543
:100520003F07A604280C9B0A54068E0A1F07860460
:100530003F07A605180C5F06080C7F068707A90A67
:100540000706A60A5406A80A180CA90A5406A40A03
:10055000280C1F06EF0E3F06DF0EDF06080C060014
:1005600000081F0786043F07A604380C9D0A4704AD
:100570006704000F43063008010F43063108030FDC
:1005800043063208010F43063308070F43063608B7
:10059000010F43063708150F43063808010F4306BD
:1005A0003908030F43063A080E0F430634082C0F90
:1005B00043063B08010F43063C08030F43063D0872
:1005C000040F43063E08090F43063F086705390F2D
:1005D00043060308010F43060D0867044705FF089B
:1005E00004020F0E0C0F43073A0B0B02B709470624
:1005F000F90B67066A07FE0A3500350C4A075C0AE4
:100600006A071A0B0F0E2A00050900028F01430624
:10061000A3044306280A00022F00D406110BD405B8
:10062000FB0B03094306110BA304280A0A0220004E
:1006300040001D0B6706380B0F0E2A00050900024B
:100640008F014307A3044307820AC306290BC3058E
:10065000FB0B310C2600070C2E006F000400EF038B
:100660002F0BEE022D0B6600C304A404A304820A20
:100670008001210B0B02F90F4306160B0A027D0FB6
:100680004306510B010F43064E0B0A02070ED5011C
:10069000B7094706F90B6A071A0B020B0A02070E85
:1006A0004B0BEB0003046B034B033500F90B800786
:1006B000F90B8003F00EA4043B010F0F650B8809B2
:1006C00000020F0EA4043B01F00F5B013B002F0062
:1006D000A4055B014306700BBF0667054605730B57
:1006E000BF06670446040F025C0143067E0B1F062B
:1006F0007C0B080C0600A6058605800B1F068604E9
:100700000F025D014306890B3F06A6053F07E7057B
:10071000F90B3F06A604E704F90B1406970BFA063B
:10072000990B07079D0B0704B40B14068F0BFA06F1
:10073000910B07069D0B0705B40BA70440031E0E83
:1007400028008006080534070804340788090802D1
:100750004306BA0BFD0E4306B40B9406F90BA30433
:10076000780B080C0600660006042604A4047A0030
:10077000BA027C006900F90B740403077405340C99
:1007800020001402020BB4040307B405340C20004B
:100790001402020B0C023A000002120F4306FA0484
:1007A000010F4306FA053A0C20001A02020B000260
:1007B0003F0F4307F90BA402E006E60B1406E80B13
:1007C000FA06EA0B0707EE0B0704B40B1406E00B5E
:1007D000FA06E20B0706EE0B0705B40B00032F0029
:1007E0000F0328004003290034059F06A70BA70527
:0C07F000F90BD404C304A304A404820A7F
:0207FE00700C7D
:021FFE00E60FEC
:00000001FF
